:0200000041C0FD
:10000200FECFFDCFFCCFFBCFFACFF9CFF8CFF7CFA2
:10001200F6CFF5CFF4CFF3CFF2CFF1CFF0CFEFCFD2
:10002200EECFEDCF1027E80364000A0001000010B4
:100032000001100001006400C80090012003F8FFD5
:10004200FCFFFEFFFFFF54656D702E3D20002D006A
:100052002532642E0025642043656C736975730D27
:1000620000427573206572726F72200A0D000100E2
:100072002D4E414E00494E46000001009300700093
:100082000000F894EE27ECBBE5BFF8E1A4B7A77F28
:10009200A4BFF1BDE1BD8DE0A2E0ED938A95E9F741
:1000A20080E8A0E6ED938A95E9F7ECE7F0E0859128
:1000B2009591009761F0A591B59105901590BF01BA
:1000C200F00105900D920197E1F7FB01F0CFE0E01E
:1000D200E3BBE4BBE5BBEFEDEDBFC0E886C00ED3EA
:1000E20018E01130C8F0EA81AB81AE27E1E0EA23E3
:1000F2000E2F003011F404D207C0AB81E8E1EA27E9
:10010200EB83FED1EB83E068EB83EA81FED1F595C8
:10011200E795EA831150E5CFEB81F7D22496089553
:10012200F6D1E4E4EA9378D2E2E0F0E0F4D122D22C
:10013200EED1EEEBEA9370D23324E9E03E1678F486
:10014200E32DE757EF9363D2AF91EC935A92A9E86C
:10015200A30DEC91EA93C3DF5E2E3394EECF5520CC
:1001620009F03FC0E0918A00E295E07F6E2FA091F6
:100172008900B0E0E0E1F0E09DD2E62B4E2EB09196
:100182008A00A0E0E0918900C0D1F070EA2BFB2B3D
:100192003F01E8E4F0E0C2D177FE0AC0E0E5F0E01A
:1001A200BDD1EFEFFFEF6E267F26F30131963F01BF
:1001B200E2E5F0E0B0D1F30146D2A7D1FF276627EE
:1001C2007727B1D1E7E5F0E0A6D1F301EF70F07047
:1001D200F695E795ADE7B0E04AD266277727A3D137
:1001E20003C0E3E6F0E09AD10895E0E8E6BDE0E07E
:1001F200E6BDE0E1E8BBEFE1E7BBE2E0E2BBE1BB89
:10020200E0E0EBBFE5BFE9BFEDB9EBB9E8E1EAB980
:10021200E6E0E3B9E0E0E2B9EFE2E9B9B7D1E1E063
:100222003E2EE5E03E1660F4E32D6FD13197A8E053
:10023200B0E000D2EF707CD1E0E17AD13394F1CF1B
:100242006FDFE4E6F0E067D195D1FACFFFCF5D9B97
:10025200FECFE881ECB921960895E981EA93F7DFB0
:10026200A881ED91FD913196FE93EE932296089529
:10027200269740D210E0AC85E0E0F0E0ED93FC93ED
:10028200E889F9893196E88BF98B3197E4912E2F21
:10029200E03009F400C1E12FE03031F4253211F4ED
:1002A20011E001C04AD1F6C0E130A1F4253211F4C7
:1002B20044D1EFC012E040E000E02D3211F401E041
:1002C200E9C02B3211F44BE2E5C0203211F440E2D6
:1002D200E1C002C0E23039F450E013E0203311F4FF
:1002E2000068D8C003C0E33009F0D4C0203310F056
:1002F2002A3308F008C0E52FAAE0AED15E2FE22F24
:10030200E0535E0FC7C0E22FE33631F41DD1EF8513
:10031200A481AA931DD1BDC0E33741F415D11ED1EA
:10032200EC91EE83EA93D8D01E2F0BC0E03769F42C
:100332000BD114D1D2D115D117D1EDD0D6D01E2FD9
:10034200086002600F7730E030C0E43611F0E93621
:1003520011F4046002C0E53729F4E6E2F0E001D1CD
:1003620015E00BC0E83511F4086003C0E83709F066
:1003720090C0E0E3F0E0F5D014E002FF12C0E4D058
:10038200EDD0ABD1F4D0AB85AA232AF4EA85FB8564
:100392004DD1EDD04DE2403011F01F5F01C00B7F17
:1003A20004C0D2D0DBD099D1E2D000FD10C0151725
:1003B20070F407FF08C002FF04C00B7F242F115006
:1003C20001C020E301C020E2B8D05150F0CF312F5C
:1003D20001FF12C0303079F003FF04C0C5D025916F
:1003E200C0D003C0AE812D91AE83A7D0503009F0AA
:1003F20051503150EFCF44C020E3B6D072D1E887DC
:10040200F987B2D03296ADD0E885F985AA85BB8549
:10041200AE17BF0748F02F5FA885B985EA85FB852F
:10042200EA1BFB0BA4D0F0CF2A3328F003FF02C053
:10043200295F01C0295D04FD19C0213320F4A8857C
:10044200B985119709F409C0531710F000FF01C0D4
:1004520011C020E207FF0AC020E3006102FF06C0CC
:100462000B7F4A9375D0503009F0515066D050300E
:1004720009F051503150A885B985129708F0BCCFC8
:1004820000FF07C0503029F05150E0E2EA9360D0FB
:10049200F9CF10E0F5CEAC8520D133D16296089524
:1004A200FF92F82E24971A93AC2FAF5FAF0D1A2F3D
:1004B200E0E0EB83EC83AC2FAB5FAF0D0ED12BD022
:1004C2001A93EEE2F1E027D0EC2FEA5FEA93D0DE56
:1004D20018812596FF900895BB27A991EE276D916B
:1004E200662311F0E395FBCF0895AA27BB27E99174
:1004F200F9910590002011F01196FBCFFD010895AE
:10050200EB81F0E0F595E7950895F0E008953ED08F
:10051200ECECEA9381C0FA93EA930895FCDF80E061
:10052200BFDF22960895E1D084E0BADF26960895CF
:10053200E8BBE8EEF3E0EFDF1DC02A93ED85EA9316
:10054200EF85F88909950895EF85E450EF870895BE
:10055200ED85EA93EF85F88909950895AF85AC5F3B
:100562000895EE83FF830895EE81FF810895EA875F
:10057200FB870895E991F991309639F083E397E08A
:100582000197F1F7A8953197C9F70895EE27939847
:100592008B9A85E793E00197F1F78B9882E28A952F
:1005A200F1F7839B08958BEB8A95F1F7839BE1E04A
:1005B2008FEC92E00197F1F708958B9A85E08A9586
:1005C200F1F78B988BE18A95F1F7889483990894D7
:1005D200E79585EC8A95F1F70895E8948B9A85E082
:1005E2008A95F1F770FD8B9880E28A95F1F78399ED
:1005F20003C070FF03C0089570FF089588EB8A95C9
:10060200F1F78B988CE08A95F1F76894089568E089
:10061200D4DF6A95E9F7089568E07991EE27DDDF86
:1006220026F477956A95D9F7E3950895F195E195C2
:10063200F0400895EE230E2EFD0121F0F695E79588
:100642000A94E1F70895F695E795F695E795F695FC
:10065200E795F695E79508950A2EAA1BB9E003C01F
:1006620008F4A00DA695E795BA95D1F708950A2E3C
:100672001B2E81E1AA27BB1B05C010F4A00DB11DE2
:10068200B695A795F795E7958A95B9F70895002449
:10069200112490E1AA0FBB1F001C111C0E1A1F0A85
:1006A20018F40E0E1F1E01C0A1609A9599F7FD0164
:1006B200D001089504D0EBDF0EF4B8DF0895E8947A
:1006C200F7FF02C0B3DF6894B7FF06C0A095B095EC
:1006D200119600F8039400FA0895ED91FC91AA9501
:1006E20008950590F491E02D08957A936A93FA9310
:1006F200EA9308955A934A933A932A931A930A9340
:1007020008955D814C813B812A8119810881089578
:00000001FF
